:103800000C94341C0C944F1C0C944F1C0C944F1CA7
:103810000C944F1C0C944F1C0C944F1C0C944F1C7C
:103820000C944F1C0C944F1C0C944F1C0C944F1C6C
:103830000C944F1C0C944F1C0C944F1C0C944F1C5C
:103840000C944F1C0C944F1C0C944F1C0C944F1C4C
:103850000C944F1C0C944F1C0C944F1C0C944F1C3C
:103860000C944F1C0C944F1C11241FBECFEFD4E0BE
:10387000DEBFCDBF11E0A0E0B1E0EAEAFFE302C0A5
:1038800005900D92A030B107D9F712E0A0E0B1E0A9
:1038900001C01D92A434B107E1F70C94991F0C9458
:1038A000001C0F93EF93FF9340D0FC01062F36D0FE
:1038B000FF91EF910F9108950F930F921F92EF9345
:1038C000FF9333D0FC010B0101E028D0FF91EF9171
:1038D0001F900F900F9108950F930F92EF93FF9306
:1038E00024D0FC0160FD60935700C895802DE395BE
:1038F000C895902DFF91EF910F900F9108950F9320
:103900000F9213D0082E09E009D00F900F9108955F
:103910000F930BD001E102D00F910895F999FECFDA
:1039200000935700E895FFFF00000091570000FD4D
:10393000FCCF08958AE08093C4008091C10080612B
:103940008093C1008091C10088608093C100089578
:103950008091C6009927089540E050E04817590724
:1039600050F423EC39E000002150304037FFFBCF0A
:103970004F5F5F4FF3CF08958091C0009927807803
:10398000907008958091C1008F7E8093C1008091D6
:10399000C100877F8093C10008950E94C21C0C94CF
:1039A000000008958093C6008091C00086FFFCCF80
:1039B0008091C00080648093C00008950E94BC1C68
:1039C0008823E1F30E94A81C803219F481E090E082
:1039D000089585E10E94D21C80E090E0089508954A
:1039E000EF92FF920F931F93CF93DF937B01C0E081
:1039F000D0E0C617D70770F48C010E94BC1C882346
:103A0000E1F30E94A81CF80181938F012196CE1545
:103A1000DF0598F381E090E0DF91CF911F910F9146
:103A2000FF90EF90089590E0282F3327213831053B
:103A300089F02238310524F42038310549F00DC0D1
:103A40002238310549F02839310539F493E005C0B1
:103A500092E003C091E001C092E1892F9927089577
:103A600040E050E0609140017091410146175707D6
:103A7000E8F4E2E4F1E08091420281BD80914202EB
:103A800090914302292F332722BD01969093430240
:103A900080934202808180BDFA9AF99AF999FECF0B
:103AA0004F5F5F4F31964617570728F308950F93DE
:103AB0001F93CF93DF9300E010E08091400190913D
:103AC000410108171907D8F4C2E4D1E080914202FD
:103AD00090914302880F991F60E0800F911F0E9410
:103AE0006C1C8883892F992789830E5F1F4F22962C
:103AF00080914001909141010817190738F3DF9137
:103B0000CF911F910F9108958091400190914101B3
:103B10000097C1F0E2E4F1E0AC018091420281BD86
:103B20008091420290914302292F332722BD0196B2
:103B30009093430280934202F89A80B5819341505A
:103B4000504059F708950F931F93CF93DF938C0143
:103B50006115710541F0EB01F80181918F010E941F
:103B6000D21C2197C9F781E090E0DF91CF911F919E
:103B70000F910895EF92FF920F931F93CF93DF93CE
:103B8000C0E0D0E08E017E01CFE7D0E0F0924302AA
:103B9000E092420263E0C8010E94511C219780E438
:103BA00090E0E80EF91E00581F4FD7FFEFCF0E949C
:103BB000881CDF91CF911F910F91FF90EF90089596
:103BC000EF92FF920F931F93CF93DF9300E010E0EB
:103BD00080914001909141010817190708F047C0F2
:103BE000EE24FF24E801CD5BDE4FF801EE5BFE4FD3
:103BF000EE0DFF1D4081888122969927382F2227BC
:103C0000240F311D8091420290914302880F991F29
:103C1000B9018E0D9F1D0E945C1C82E090E0E80EB1
:103C2000F91E90E8E916F10400F3809142029091A8
:103C30004302880F991F63E0800F911F0E94511C5F
:103C40008091420290914302880F991F65E0800F96
:103C5000911F0E94511C0E94881C00581F4F809188
:103C60004001909141010817190708F4B9CFDF917D
:103C7000CF911F910F91FF90EF900895CF93C0E0E7
:103C800069E081E090E00E946C1C84FF03C08F7E9D
:103C90000E947F1C0E94BC1C8823E1F30E94A81C88
:103CA000992782359105DCF4803591050CF054C0DC
:103CB0008134910509F45AC0823491053CF4803373
:103CC000910509F449C0C19759F12FC1823491057A
:103CD00009F45FC08534910509F45EC026C18635BC
:103CE000910509F4EDC0873591054CF482359105B5
:103CF00009F461C08535910509F465C016C18437A2
:103D0000910509F4A0C0853791052CF484369105FE
:103D100009F472C00AC18537910509F4C1C005C113
:103D20000E94DE1C882309F4B5CF84E10E94D21CD6
:103D300081E40E94D21C86E50E94D21C82E50E948A
:103D4000D21C80E20E94D21C83E50E94D21C84E532
:103D50000E94D21C8BE406C00E94DE1C882309F45A
:103D600099CF84E10E94D21C80E1E0C061E070E064
:103D700080E091E00E94F01C0E94DE1C882309F480
:103D800089CF84E10E94D21C809100010E94131D02
:103D9000E9CF64E170E00AC061E070E080E091E0AA
:103DA0000E94F01C809100019927BC0180E091E005
:103DB0000E94F01CD1CF0E94DE1C882309F46ACF38
:103DC0000E94BA1DCECF62E070E080E091E00E94D8
:103DD000F01C0E94DE1C882309F45CCF20910001B6
:103DE000809101019927982F8827820F911D909328
:103DF000430280934202B5CF63E070E080E091E03F
:103E00000E94F01C20910101809100019927982FB8
:103E10008827820F911D9093410180934001BC013E
:103E200082E491E00E94F01C0E94DE1C882309F4C9
:103E300031CF80910201863419F40E94E01D91CFA8
:103E40000E94301D8ECF63E070E080E091E00E9420
:103E5000F01C20910101809100019927982F88275B
:103E6000820F911D90934101809340010E94DE1CBE
:103E7000882309F40FCF80910201863419F40E943F
:103E8000571D02C00E94841D84E10E94D21C6091D3
:103E900040017091410182E491E00E94A31D64CF32
:103EA0000E94DE1C882309F4F5CE84E10E94D21C16
:103EB0008EE10E94D21C84E90E94D21C86E052CF7F
:103EC00064E070E080E091E00E94F01C0E94DE1C43
:103ED000882309F4DFCE84E10E94D21C8091000186
:103EE000803531F480910101882361F4C82F17C017
:103EF000883531F480910101883061F4C3E00FC04E
:103F0000803531F480910101883049F4C2E007C066
:103F1000883529F480910101882309F4C1E069E022
:103F20008C2F99270E946C1C1DCF85E10E94D21C0A
:103F3000B1CECFEFD4E0DEBFCDBFCEE1F8948EEFAF
:103F400091E00E94CC1F843B61F48FEF91E00E94CE
:103F5000CC1F833C31F48DEF91E00E94CC1F809305
:103F600066000E949A1C0E94A81C84E690E00E94B1
:103F7000AC1C0E94BC1C882321F4C150C5B9CC23C1
:103F8000A1F7CC2319F00E943E1E02C00E94CD1C56
:103F900080E090E00C94D41FE199FECF9FBB8EBBD4
:0A3FA000E09A99278DB30895FFCF32
:0400000300003800C1
:00000001FF
